:1000000012C12AC129C128C1B8C126C125C190C1C8
:1000100060C122C121C13BC21FC1EDC11DC11CC1B4
:100020001BC11AC119C100C0C101C30302C2C60667
:1000300007C705C5C404CC0C0DCD0FCFCE0E0ACA20
:10004000CB0BC90908C8D81819D91BDBDA1A1EDE70
:10005000DF1FDD1D1CDC14D4D515D71716D6D21220
:1000600013D311D1D010F03031F133F3F23236F630
:10007000F737F53534F43CFCFD3DFF3F3EFEFA3AE0
:100080003BFB39F9F83828E8E929EB2B2AEAEE2E70
:100090002FEF2DEDEC2CE42425E527E7E62622E2E0
:1000A000E323E12120E0A06061A163A3A26266A630
:1000B000A767A56564A46CACAD6DAF6F6EAEAA6AA0
:1000C0006BAB69A9A86878B8B979BB7B7ABABE7EF0
:1000D0007FBF7DBDBC7CB47475B577B7B67672B2A0
:1000E000B373B17170B05090915193535292965630
:1000F0005797559594549C5C5D9D5F9F9E5E5A9A60
:100100009B5B99595898884849894B8B8A4A4E8EEF
:100110008F4F8D4D4C8C448485458747468682425F
:1001200043834181804000C1814001C0804101C0C2
:10013000804100C1814001C0804100C1814000C1B7
:10014000814001C0804101C0804100C1814000C1A7
:10015000814001C0804100C1814001C0804101C097
:10016000804100C1814001C0804100C1814000C187
:10017000814001C0804100C1814001C0804101C077
:10018000804100C1814000C1814001C0804101C067
:10019000804100C1814001C0804100C1814000C157
:1001A000814001C0804101C0804100C1814000C147
:1001B000814001C0804100C1814001C0804101C037
:1001C000804100C1814000C1814001C0804101C027
:1001D000804100C1814001C0804100C1814000C117
:1001E000814001C0804100C1814001C0804101C007
:1001F000804100C1814001C0804100C1814000C1F7
:10020000814001C0804101C0804100C1814000C1E6
:10021000814001C0804100C1814001C0804101C0D6
:10022000804100C1814011241FBECFEDCDBF10E041
:10023000A0E6B0E0ECE3F7E002C005900D92A03735
:10024000B107D9F720E0A0E7B0E001C01D92AE3AB7
:10025000B207E1F702D070C2D3CEA89584B7877FEA
:1002600084BF81B5886181BD8EE081BD12B886E210
:1002700089B98AB188698AB983B1866083B984E112
:1002800090E09BBD8ABD1FBC95E09EBD12BC1DBC0D
:100290001CBC89B7806489BF8BEB86BF10BE93BF3F
:1002A00012BE89B7816089BF8BB780628BBF80B572
:1002B000876080BD88E187BB8A9A929882B38867FD
:1002C00082BB80B385E8809399007894C39A00003C
:1002D000FECF1F920F920FB60F9211248F939F9310
:1002E000EF93FF939091710080917200891750F401
:1002F00092988AB1877D8AB9C49810927100109241
:1003000072000DC0929AC49AE091710081E08E0F44
:1003100080937100F0E0EB57FF4F80818CB9FF9123
:10032000EF919F918F910F900FBE0F901F90189596
:100330001F920F920FB60F9211248F93EF93FF939A
:100340005F9B13C0C39AE0917000E43148F481E0F0
:100350008E0F809370008CB1F0E0E656FF4F8083E3
:10036000C3981DBC1CBC85E08EBDFF91EF918F91A1
:100370000F900FBE0F901F9018951F920F920FB6FF
:100380000F9211242F933F934F935F936F937F931B
:100390008F939F93AF93BF93EF93FF938EB58A7F15
:1003A0008EBD809170008823A9F08091810090918A
:1003B0008200892B09F0C39AFED0882359F010924D
:1003C000700010927E0010927D00109282001092B8
:1003D0008100C398FF91EF91BF91AF919F918F9151
:1003E0007F916F915F914F913F912F910F900FBE31
:1003F0000F901F9018951F920F920FB60F92112415
:100400002F933F934F935F936F937F938F939F931C
:10041000A895209181003091820080917B0090917D
:100420007C00232B79F421E030E04091740050915E
:1004300075008417950714F020E030E030938400B5
:1004400020938300909375008093740080917600D0
:10045000909177006CE370E05ED124E096958795EB
:100460002A95E1F79093800080937F0010927700A7
:10047000109276009F918F917F916F915F914F9134
:100480003F912F910F900FBE0F901F9018951F92C4
:100490000F920FB60F9211242F933F934F936F93A8
:1004A0007F938F939F93EF93FF9346B34370E091B5
:1004B0007300F0E0EE0FFF1FEE0FFF1FE05AFF4F3B
:1004C000E40FF11D8081082E000C990B20917B0018
:1004D00030917C00280F391F30937C0020937B00E3
:1004E00060917D0070917E00860F971F90937E0033
:1004F00080937D004093730086B38770813049F408
:100500008091760090917700019690937700809388
:100510007600C9018150904F8F3F9F4110F4232BEB
:1005200051F410927C0010927B0081E090E0909357
:10053000820080938100FF91EF919F918F917F9135
:100540006F914F913F912F910F900FBE0F901F9081
:100550001895DC01680F791F9FEF4FEF2D919227BF
:10056000292F30E0F901EA5DFE4F94919427F901BB
:10057000EA5DFF4F44916A177B0781F7892F90E06E
:10058000942B0895CF93DF93C5E8D0E09091990024
:100590009883806889836A8363E070E0CE01D9DF45
:1005A0009C838B8385E0809372008AB188628AB9CC
:1005B000DF91CF9108950F931F93CF93DF936091B5
:1005C0007000683008F49BC090919A008091990067
:1005D000981395C0C0919B00C43021F0C63009F437
:1005E0006CC08FC00091A0001091A10070E062501B
:1005F00071098AE990E0ADDF8017910711F063E09F
:1006000081C080919E0090919F009827892798270C
:100610009C01215031092630310508F070C020912D
:100620009C0030919D00182F110F4091990040932C
:100630008500C093860010938700232BD9F5FC0119
:10064000EE0FFF1FE857FF4F0197DC01AA0FBB1FFA
:10065000A758BF4F2D913C91329737FF03C031957A
:1006600021953109322723273227318320830097B0
:1006700059F72091790030917A0081E090E0232BA6
:1006800011F080E090E090937A0080937900C12F80
:10069000D0E02396BE0185E890E05BDFCB57DF4FCB
:1006A000998388831B5F109372008AB188628AB92C
:1006B00081E02CC062E084E027C0E0919E00F091D0
:1006C0009F00FE27EF27FE27CF0101970697B8F47A
:1006D000EE0FF0E0E656FF4FC581D0E0DC2FCC27CF
:1006E0008481C82B70E0625071098AE990E031DFA3
:1006F000C817D90709F083CF62E086E005C060E043
:1007000001C061E080919B003DDF80E0DF91CF91EF
:100710001F910F9108950024552704C0080E591FFA
:10072000880F991F009729F076956795B8F37105A2
:0C073000B9F7802D952F0895F894FFCFA5
:10073C0000FF0100010000FFFF0000010001FF00AD
:00000001FF
